:0200000480007A
:100000006F008004732F2034930F80006308FF0378
:10001000930F90006304FF03930FB0006300FF038E
:10002000130F000063040F0067000F00732F2034CC
:1000300063540F006F00400093E19153171F0000BD
:1000400023223FFC6FF09FFF93000000130100008C
:10005000930100001302000093020000130300004C
:100060009303000013040000930400001305000034
:10007000930500001306000093060000130700001C
:100080009307000013080000930800001309000004
:1000900093090000130A0000930A0000130B0000EC
:1000A000930B0000130C0000930C0000130D0000D4
:1000B000930D0000130E0000930E0000130F0000BC
:1000C000930F0000732540F16310050097020000B4
:1000D000938202017390523073500018970200000F
:1000E0009382020273905230B70200809382F2FF33
:1000F0007390023B9302F0017390023A73504030C8
:100100009702000093824201739052307350203066
:100110007350303093010000970200009382C2EECA
:1001200073905230130510001315F501634C050050
:100130000F00F00F930110009308D0051305000085
:100140007300000093020000638A02007390521053
:10015000B7B2000093829210739022307350003037
:10016000970200009382420173901234732540F18C
:1001700073002030972000009380C0E83701AA0068
:100180001301A10A23A0200003A70000B703AA00BF
:100190009383A30A93012000631077469720000001
:1001A000938040E637B100AA130101A023A22000EA
:1001B00003A74000B7B300AA938303A093013000C4
:1001C000631C7742972000009380C0E33711A00A98
:1001D000130101AA23A4200003A78000B713A00ADB
:1001E000938303AA9301400063187740972000008F
:1001F000938040E137A10AA01301A10023A62000AB
:1002000003A7C000B7A30AA09383A30093015000E3
:100210006314773E97200000938080E03701AA00A6
:100220001301A10A23AA20FE03A740FFB703AA00D7
:100230009383A30A930160006310773C972000002A
:10024000938000DE37B100AA130101A023AC20FE89
:1002500003A780FFB7B300AA938303A093017000A4
:10026000631C773897200000938080DB3711A00A49
:10027000130101AA23AE20FE03A7C0FFB713A00AF3
:10028000938303AA930180006318773697200000B8
:10029000938000D937A10AA01301A10023A0200058
:1002A00003A70000B7A30AA09383A30093019000C3
:1002B00063147734972000009380C0D637513412EE
:1002C00013018167138200FE2320220283A2000013
:1002D000B7533412938383679301A000639E7230F7
:1002E00097200000938000D43731215813018109F1
:1002F0009380D0FFA3A32000172200001302C2D2D4
:1003000083220200B7332158938383099301B000FD
:100310006394722E9301C00013020000B7D0BBAAF1
:100320009380D0CD172100001301C1CD23201100EF
:1003300003270100B7D3BBAA9383D3CD631E772ACB
:100340001302120093022000E31A52FC9301D00022
:1003500013020000B7C0ABDA9380D0CC17210000A5
:10036000130141CA1300000023221100032741009A
:10037000B7C3ABDA9383D3CC631077281302120090
:1003800093022000E31852FC9301E00013020000E6
:10039000B7C0AADD9380C0BC17210000130181C63D
:1003A0001300000013000000232411000327810024
:1003B000B7C3AADD9383C3BC631077241302120072
:1003C00093022000E31652FC9301F0001302000098
:1003D000B7B0DACD9380C0BB130000001721000036
:1003E000130141C2232611000327C100B7B3DACDA0
:1003F0009383C3BB63127720130212009302200081
:10040000E31852FC9301000113020000B7B0DDCCE9
:100410009380B0AB1300000017210000130181BED0
:10042000130000002328110003270101B7B3DDCC1E
:100430009383B3AB6312771C130212009302200064
:10044000E31652FC9301100113020000B7E0CDBC8B
:100450009380B0AA130000001300000017210000D1
:10046000130141BA232A110003274101B7E3CDBC90
:100470009383B3AA63127718130212009302200029
:10048000E31652FC93012001130200001721000023
:10049000130141B7B72011009380302323201100AE
:1004A00003270100B72311009383332363167714C6
:1004B0001302120093022000E31A52FC9301300150
:1004C00013020000172100001301C1B3B71001305F
:1004D00093803022130000002322110003274100E3
:1004E000B71301309383332263187710130212007D
:1004F00093022000E31852FC930140011302000014
:1005000017210000130101B0B710003393802012AF
:1005100013000000130000002324110003278100B2
:10052000B7130033938323126318770C130212005E
:1005300093022000E31652FC9301500113020000C5
:1005400017210000130101AC13000000B700302395
:1005500093802011232611000327C100B703302305
:1005600093832311631A7708130212009302200069
:10057000E31852FC930160011302000017210000F0
:10058000130141A813000000B7003322938010012B
:10059000130000002328110003270101B7033322B1
:1005A00093831301631A770413021200930220004D
:1005B000E31652FC930170011302000017210000A2
:1005C000130141A41300000013000000B7302312F0
:1005D00093801000232A110003274101B73323120F
:1005E00093831300631A7700130212009302200012
:1005F000E31652FC631030020F00F00F638001001D
:100600009391110093E111009308D0051385010027
:10061000730000000F00F00F930110009308D00545
:100620001305000073000000731000C000000000FC
:0C063000000000000000000000000000BE
:1010000000000000000000000000000000000000E0
:1010100000000000000000000000000000000000D0
:1010200000000000000000000000000000000000C0
:1010300000000000000000000000000000000000B0
:081040000000000000000000A8
:10200000EFBEADDEEFBEADDEEFBEADDEEFBEADDEF0
:10201000EFBEADDEEFBEADDEEFBEADDEEFBEADDEE0
:10202000EFBEADDEEFBEADDE000000000000000040
:040000058000000077
:00000001FF
